:06000000020033020E664F
:03000B00020E677B
:03001300020E8159
:03001B00020E8250
:03002300020E8347
:03002B00020E843E
:10003300759840758780758921758DFF758BFF7560
:100043008850D299758160758CFA758A0075A8827B
:1000530075900075B0FF7535FF7537FF7539FF75FE
:100063003BFF753DFF753FFF7541FF7543FF7545C9
:10007300FF753600753800753A00753C00753E0013
:1000830075400075420075440075300C753100D21F
:10009300A0D2A1782076FF08B830FAC2A27E80DF12
:1000A300FEDEFCC280C287C286D285D284D2A3C2BE
:1000B300A3DFFEDFFEDFFEDFFEDFFED2A3C2A3DF90
:1000C300FED2A3C2A3DFFEC284D2A3C2A3742812AA
:1000D30010BFDFFE74081210BFDFFE74061210BFDC
:1000E300DFFE74101210BFDFFE740C1210BFDFFEB0
:1000F30074011210BFDFFEDFFE74401210BF7F4099
:10010300901358E4931210E4A3DFF874801210BF25
:100113007F14901398E4931210E4A3DFF874C012D1
:1001230010BF7F149013ACE4931210E4A3DFF8DF45
:10013300FEDEFCDFFEDEFCDFFEDEFCDFFEDEFC744B
:10014300801210BF7F149013C0E4931210E4A3DF56
:10015300F874C01210BF7F149013D4E4931210E408
:10016300A3DFF8759000D2A0D2A17880E670257540
:10017300B0FE75A00120A00F300019C200760890D0
:1001830011CC120F25800D20000AD20076089011A1
:10019300CF120F257881E6702575B0FE75A0022079
:1001A300A10F300119C20176089011D2120F2580D8
:1001B3000D20010AD20176089011D5120F257890EF
:1001C300E6702575B0FB75A00120A00F301019C291
:1001D3001076089011D8120F25800D20100AD21026
:1001E30076089011DB120F257891E6702575B0FB28
:1001F30075A00220A10F301119C21176089011DEEB
:10020300120F25800D20110AD21176089011E112E8
:100213000F257898E6702575B0F775A00120A00F1B
:10022300301819C21876089011E4120F25800D209A
:10023300180AD21876089011E7120F257899E670FC
:100243002575B0F775A00220A10F301919C21976D0
:10025300089011EA120F45800D20190AD219760869
:100263009011ED120F4578A0E6702575B0EF75A0DB
:100273000120A00F302019C22076089011F0120F30
:1002830025800D20200AD22076089011F3120F2525
:1002930075B0EF75A00220A126753207120E9312D6
:1002A3000E85D53206753201120E93120E8C75B07F
:1002B300EF75A00220A10820190302119580E378AD
:1002C300A8E6702575B0DF75A00120A00F302819AE
:1002D300C22876089011F6120F25800D20280AD225
:1002E3002876089011F9120F2575B0DF75A002204A
:1002F300A126753207120EB8120E85D53206753255
:1003030001120EB8120E8C75B0DF75A00220A10881
:1003130020190302119580E378B0E6702575B0BF0C
:1003230075A00120A00F303019C23076089011FC5F
:10033300120F25800D20300AD23076089011FF125B
:100343000F2575B0BF75A00220A120753207120ECC
:10035300DD120E85D53206753201120EDD120E8CBA
:1003630075B0BF75A00220A10280E978B8E67025B8
:1003730075B07F75A00120A00F303819C2387608F8
:10038300901202120F25800D20380AD23876089079
:100393001205120F2575B07F75A00220A1207532BA
:1003A30007120F01120E85D53206753201120F01A5
:1003B300120E8C75B07F75A00220A10280E97590A2
:1003C300FFC2A0C2A178C0E6702575B0FE7590018A
:1003D30020900F304019C2407608901208120F2562
:1003E300800D20400AD240760890120B120F257818
:1003F300C1E6702575B0FE75900220910F3041194A
:10040300C241760890120E120F25800D20410AD2A8
:10041300417608901211120F2578C2E6702575B047
:10042300FE75900420920F304219C2427608901252
:1004330014120F25800D20420AD24276089012171B
:10044300120F2578C3E6702575B0FE7590082093CA
:100453000F304319C243760890121A120F25800DEC
:1004630020430AD243760890121D120F2578C4E662
:10047300702575B0FE75901020940F304419C24456
:100483007608901220120F25800D20440AD244765C
:1004930008901223120F2578C5E6702575B0FE75F6
:1004A300902020950F304519C245760890122612E8
:1004B3000F25800D20450AD2457608901229120F88
:1004C3002578C6E6702575B0FE75904020960F30EE
:1004D3004619C246760890122C120F25800D20462D
:1004E3000AD246760890122F120F2578C7E6702598
:1004F30075B0FE75908020970F304719C247760874
:10050300901232120F25800D20470AD247760890A9
:100513001235120F2578D0E6702575B0FB75900162
:1005230020900F305019C2507608901238120F25C0
:10053300800D20500AD250760890123B120F257876
:10054300D1E6702575B0FB75900220910F305119DB
:10055300C251760890123E120F25800D20510AD207
:10056300517608901241120F2578D2E6702575B0A6
:10057300FB75900420920F305219C25276089012E4
:1005830044120F25800D20520AD25276089012474A
:10059300120F2578D3E6702575B0FB75900820936C
:1005A3000F305319C253760890124A120F25800D4B
:1005B30020530AD253760890124D120F2578D4E6B1
:1005C300702575B0FB75901020940F305419C254E8
:1005D3007608901250120F25800D20540AD25476BB
:1005E30008901253120F2578D5E6702575B0FB7568
:1005F300902020950F305519C25576089012561247
:100603000F25800D20550AD2557608901259120FE6
:100613002578D6E6702575B0FB75904020960F308F
:100623005619C256760890125C120F25800D20567B
:100633000AD256760890125F120F2578D7E67025F6
:1006430075B0FB75908020970F305719C257760805
:10065300901262120F25800D20570AD25776089008
:100663001265120F2578D8E6702575B0F7759001DD
:1006730020900F305819C2587608901268120F252F
:10068300800D20580AD258760890126B120F2578E5
:10069300D9E6702575B0F775900220910F3059197E
:1006A300C259760890126E120F25800D20590AD276
:1006B300597608901271120F2578DAE6702575B015
:1006C300F775900420920F305A19C25A7608901287
:1006D30074120F25800D205A0AD25A760890127789
:1006E300120F2578DBE6702575B0F7759008209317
:1006F3000F305B19C25B760890127A120F25800DBA
:10070300205B0AD25B760890127D120F2578DCE617
:10071300702575B0F775901020940F305C19C25C8A
:100723007608901280120F25800D205C0AD25C7629
:1007330008901283120F2578DDE6702575B0F775E2
:10074300902020950F305D19C25D760890128612B5
:100753000F25800D205D0AD25D7608901289120F55
:100763002578DEE6702575B0F775904020960F303A
:100773005E19C25E760890128C120F25800D205EE2
:100783000AD25E760890128F120F2578DFE6702565
:1007930075B0F775908020970F305F19C25F7608A8
:1007A300901292120F25800D205F0AD25F76089077
:1007B3001295120F2578E0E6702575B0EF7590015C
:1007C30020900F306019C2607608901298120F259E
:1007D300800D20600AD260760890129B120F257854
:1007E300E1E6702575B0EF75900220910F30611925
:1007F300C261760890129E120F25800D20610AD2E5
:100803006176089012A1120F2578E2E6702575B083
:10081300EF75900420920F306219C262760890122D
:10082300A4120F25800D20620AD26276089012A7C7
:10083300120F2578E3E6702575B0EF7590082093C5
:100843000F306319C26376089012AA120F25800D28
:1008530020630AD26376089012AD120F2578E4E67E
:10086300702575B0EF75901020940F306419C26431
:1008730076089012B0120F25800D20640AD2647698
:10088300089012B3120F2578E5E6702575B0EF7561
:10089300902020950F306519C26576089012B61224
:1008A3000F25800D20650AD26576089012B9120FC4
:1008B3002578E6E6702575B0EF75904020960F30E9
:1008C3006619C26676089012BC120F25800D206649
:1008D3000AD26676089012BF120F2578E7E67025D4
:1008E30075B0EF75908020970F306719C26776084F
:1008F3009012C2120F25800D20670AD267760890E6
:1009030012C5120F2578E8E6702575B0DF759001E2
:1009130020900F306819C26876089012C8120F250C
:10092300800D20680AD26876089012CB120F2578C2
:10093300E9E6702575B0DF75900220910F306919D3
:10094300C26976089012CE120F25800D20690AD253
:100953006976089012D1120F2578EAE6702575B0F2
:10096300DF75900420920F306A19C26A76089012DC
:10097300D4120F25800D206A0AD26A76089012D706
:10098300120F2578EBE6702575B0DF75900820937C
:100993000F306B19C26B76089012DA120F25800D97
:1009A300206B0AD26B76089012DD120F2578ECE6E5
:1009B300702575B0DF75901020940F306C19C26CE0
:1009C30076089012E0120F25800D206C0AD26C7607
:1009D300089012E3120F2578EDE6702575B0DF75E8
:1009E300902020950F306D19C26D76089012E61293
:1009F3000F25800D206D0AD26D76089012E9120F33
:100A03002578EEE6702575B0DF75904020960F309F
:100A13006E19C26E76089012EC120F25800D206EAF
:100A23000AD26E76089012EF120F2578EFE6702542
:100A330075B0DF75908020970F306F19C26F7608FD
:100A43009012F2120F25800D206F0AD26F76089054
:100A530012F5120F2578F0E6702575B0BF75900179
:100A630020900F307019C27076089012F8120F257B
:100A7300800D20700AD27076089012FB120F257831
:100A8300F1E6702575B0BF75900220910F30711992
:100A9300C27176089012FE120F25800D20710AD2C2
:100AA300717608901301120F2578F2E6702575B060
:100AB300BF75900420920F307219C272760890139A
:100AC30004120F25800D20720AD272760890130744
:100AD300120F2578F3E6702575B0BF759008209343
:100AE3000F307319C273760890130A120F25800D05
:100AF30020730AD273760890130D120F2578F4E64B
:100B0300702575B0BF75901020940F307419C2749E
:100B13007608901310120F25800D20740AD2747674
:100B230008901313120F2578F5E6702575B0BF757D
:100B3300902020950F307519C27576089013161200
:100B43000F25800D20750AD2757608901319120FA0
:100B53002578F6E6702575B0BF75904020960F3066
:100B63007619C276760890131C120F25800D207615
:100B73000AD276760890131F120F2578F7E67025B0
:100B830075B0BF75908020970F307719C2777608BC
:100B9300901322120F25800D20770AD277760890C2
:100BA3001325120F2578F8E6702575B07F7590012F
:100BB30020900F307819C2787608901328120F25E9
:100BC300800D20780AD278760890132B120F25789F
:100BD300F9E6702575B07F75900220910F30791971
:100BE300C279760890132E120F25800D20790AD230
:100BF300797608901331120F2578FAE6702575B0CF
:100C03007F75900420920F307A19C27A7608901378
:100C130034120F25800D207A0AD27A760890133782
:100C2300120F2578FBE6702575B07F759008209329
:100C33000F307B19C27B760890133A120F25800D73
:100C4300207B0AD27B760890133D120F2578FCE6B1
:100C5300702575B07F75901020940F307C19C27C7D
:100C63007608901340120F25800D207C0AD27C76E3
:100C730008901343120F2578FDE6702575B07F7534
:100C8300902020950F307D19C27D7608901346126F
:100C93000F25800D207D0AD27D7608901349120F0F
:100CA3002578FEE6702575B07F75904020960F304D
:100CB3007E19C27E760890134C120F25800D207E7C
:100CC3000AD27E760890134F120F2578FFE670251F
:100CD30075B07F75908020970F307F19C27F76089B
:100CE300901352120F25800D207F0AD27F76089031
:100CF3001355120F257590FFD2A0D2A17580FFD294
:100D0300A27407B535037535FF0535E535A2E092C5
:100D1300A4A2E192A5A2E292A6C2AFD2A7C2A7E47F
:100D2300B53503020D5604B53503020D7704B53509
:100D330003020D9804B53503020DB904B53503025A
:100D43000DDA04B53503020DFB04B53503020E1CA1
:100D5300020E3DE580F536A837A936120F6340062B
:100D630024FE500D8005120F685006853637120F8A
:100D73006F020E5EE580F538A839A938120F63407B
:100D83000624FE500D8005120F685006853839126F
:100D93000F93020E5EE580F53AA83BA93A120F6362
:100DA300400624FE500D8005120F685006853A3B1D
:100DB300120FB7020E5EE580F53CA83DA93C120F69
:100DC30063400624FE500D8005120F685006853CD3
:100DD3003D120FDB020E5EE580F53EA83FA93E12F1
:100DE3000F63400624FE500D8005120F68500685E0
:100DF3003E3F120FFF020E5EE580F540A841A94079
:100E0300120F63400624FE500D8005120F68500632
:100E1300854041121023020E5EE580F542A843A9E6
:100E230042120F63400624FE500D8005120F6850D6
:100E330006854243121077020E5EE580F544A8450D
:100E4300A944120F63400624FE500D8005120F685B
:100E5300500685444512109B020E5ED2AF02016616
:100E630002003332C0D0C0E0C0007880E6600116D3
:100E730008B800F8758CFAD000D0E0D0D032323206
:100E830032327E20DFFEDEFC227E60DFFEDEFC22CD
:100E930074801210BF05307419B53003753000E546
:100EA300307F049013E8E5302323931210E4A3DF8B
:100EB300F51211B32274801210BF153074FFB530D0
:100EC30003753018E5307F049013E8E5302323934E
:100ED3001210E4A3DFF51211B3223099FDC2997504
:100EE30099C074C01210BF3099FDC2990531748046
:100EF300B53103753100E531F59912113522309979
:100F0300FDC2997599C074C01210BF3099FDC29982
:100F1300153174FFB5310375317FE531F599121140
:100F23003522E4933099FDC299F599A3E4932530D2
:100F33003099FDC299F599A3E4933099FDC299F5CF
:100F43009922E4933099FDC299F599A3E4933099DA
:100F5300FDC299F599A3E4933099FDC299F59922BD
:100F6300C2D7E89922C2D7E99824FE223099FDC25C
:100F7300997599B074D11210BF3099FDC2997599C2
:100F83005B3099FDC299E536C313F59912113522E9
:100F93003099FDC2997599B0748D1210BF3099FDC7
:100FA300C2997599493099FDC299E538C313F599EA
:100FB300121135223099FDC2997599B074891210B6
:100FC300BF3099FDC2997599473099FDC299E53AA9
:100FD300C313F599121135223099FDC2997599B051
:100FE30074851210BF3099FDC29975994A3099FDE5
:100FF300C299E53CC313F599121135223099FDC20C
:10100300997599B074C91210BF3099FDC299759939
:10101300013099FDC299E53EC313F59912113522AA
:101023003099FDC2997599B074C51210BF3099FDFE
:10103300C2997599633099FDC2997599013099FDEB
:10104300C2997599B03099FDC2997599623099FD2D
:10105300C2997599243099FDC2997599B03099FD5B
:10106300C2997599063099FDC299E540C313F59964
:10107300121135223099FDC2997599B074911210ED
:10108300BF3099FDC2997599483099FDC299E542DF
:10109300C313F599121135223099FDC2997599B090
:1010A30074CD1210BF3099FDC29975995D3099FDC9
:1010B300C299E544C313F59912113522C2A2C28025
:1010C300339287339286339285339284D2A3C2A319
:1010D300339287339286339285339284D2A3C2A309
:1010E30022C2A2D28033928733928633928533927F
:1010F30084D2A3C2A33392873392863392853392E9
:1011030084D2A3C2A32275F0648424301210E47441
:101113000AC5F08424301210E4E5F024301210E400
:101123002275F00A8424301210E4C5F02430121022
:10113300E422D2D575F064847004C2D574F02430EF
:101143001210E4740AC5F084700520D50274F024EB
:10115300301210E4E5F024301210E42275F00A8412
:10116300700274F024301210E4E5F024301210E41D
:1011730022E493A3B45E01221210E40211747004FA
:101183007420800AC313C313C313C313C3131210EE
:10119300E4221211B33099FDC2997599B03099FDCB
:1011A300C2997599783099FDC299759900020033F7
:1011B3003099FDC2997599B03099FDC29975997BA3
:1011C3003099FDC29975990022905040805000904B
:1011D30051408051009052408052009053408053C0
:1011E30000905440805400B0407FB0400090554080
:1011F300805500905640805600905740805700908D
:101203005840805800901840801800901940801969
:1012130000901A40801A00901B40801B00901C40D5
:10122300801C00901D40801D00901E40801E009079
:101233001F40801F0090204080200090214080218B
:10124300009022408022009023408023009024407D
:101253008024009025408025009026408026009021
:10126300274080270090284080280090294080292B
:1012730000902A40802A00902B40802B00902C4025
:10128300802C00902D40802D00902E40802E0090C9
:101293002F40802F009030408030009031408031CB
:1012A30000903240803200903340803300903440CD
:1012B3008034009035408035009036408036009071
:1012C300374080370090384080380090394080396B
:1012D30000903A40803A00903B40803B00903C4075
:1012E300803C00903D40803D00903E40803E009019
:1012F3003F40803F0090404080400090414080410B
:10130300009042408042009043408043009044401C
:1013130080440090454080450090464080460090C0
:1013230047408047009048408048009049408049AA
:1013330000904A40804A00904B40804B00904C40C4
:10134300804C00904D40804D00904E40804E009068
:101353004F40804F00000000000000001F0000000D
:101363000000001F1F00000000001F1F1F000000DF
:10137300001F1F1F1F0000001F1F1F1F1F00001F34
:101383001F1F1F1F1F001F1F1F1F1F1F1F1F1F1F89
:101393001F1F1F1F1F4D757A796B616E74203720D5
:1013A30076312E30632020202020736D69616C65B7
:1013B3006B2E7072762E706C20202020202043200C
:1013C3002020313237203132372031323720313249
:1013D300372020302020313237203132372031324C
:1013E30037203132372D4320202D4465732D44207F
:1013F300202D4573202D4520202D4620202D476587
:10140300732D4720202D4173202D4120202D422074
:10141300202D482020204320202B4369732B442078
:10142300202B4469732B4520202B4620202B466913
:10143300732B4720202B4769732B4120202B4169B5
:10144300732B4820202B432020204D757A796B6124
:101453006E7420372076312E306320323030372DB2
:1014630030372D3034202863294164616D20536D5A
:1014730069616C656B206A616E6B6F6D757A796BF0
:10148300616E744077702E706C207777772E736D52
:1014930069616C656B2E7072762E706C2057737A4F
:1014A300656C6B6965207072617761207A61737412
:1014B300727A657A6F6E652E204A616B69656B6F10
:1014C3006C7769656B207A6173746F736F77616E84
:1014D3006961206B6F6D657263796A6E65206B6FEE
:1014E3006475206E6965646F7A776F6C6F6E652EB5
:1014F30020416C6C20526967687473205265736570
:10150300727665642E204672656520666F72206E62
:101513006F6E20636F6D6D65726369616C206F6EB2
:041523006C792E2091
:00000001FF
